:1000000012C0189518951895189518957EC01895D2
:100010001895189518951895189518951895189578
:100020001895189518958FED8DBFC0ECE8EB4E2E06
:10003000DD275D2EEEE7F0E0A0E6B0E0A89584B7FE
:10004000082E877F84BF88E1992781BD91BD8827CD
:100050008D933197E9F766248FEF87BB8FEF88BBCD
:100060008BEF81BB8FEF82BB80E08ABB8FEF8BBBB6
:1000700084E083BF80E080BF89B7826089BF7894C5
:1000800081E080936F000027AEE68C9186FB0EF432
:1000900001E041E0041709F00CC080916E008F7BF5
:1000A00080936E00AAE68D919C91A2E68D939C931D
:1000B000F0D00027AEE68C9185FB0EF401E041E024
:1000C000041709F01FC080916E008F7D80936E0031
:1000D0000027A0E38C9182FB0EF401E040E00417BE
:1000E00009F003C081E080936F000027A9E38C91A1
:1000F00080FB0EF401E040E0041709F003C080E04B
:1001000080936F00C0CFF894FFCF0F921F922F9271
:100110003F924F925F927F92AF92BF920F931F9345
:100120002F933F934F935F936F937F938F939F93FF
:10013000AF93BF93CF93DF93EF93FF938FB78F93DB
:1001400083E88093520080916E00806480936E00FB
:10015000A0E68C918F5F8C9300916000093109F0CB
:1001600019C080E08093600080916E00806280936F
:100170006E00A1E68C918F5F8C93009161000A3034
:1001800009F008C080E08093610080916E00806873
:1001900080936E008F918FBFFF91EF91DF91CF9190
:1001A000BF91AF919F918F917F916F915F914F918F
:1001B0003F912F911F910F91BF90AF907F905F90D3
:1001C0004F903F902F901F900F9018950027AEE60C
:1001D0008C9187FB0EF401E041E0041709F058C050
:1001E00080916E008F7780936E00AFE68C91E0E394
:1001F0005FD181E08A93AFE68C916CECBB27A6E1DE
:10020000E0E382D181E08A93AFE68C916EEBBB276D
:10021000A6E1E0E379D1AFE68C91AAE6E0E322E043
:100220002A93ACD1ABE68C9187FBAEE68C9184F936
:100230008C93AAE68D919C91CAD0AAE68D939C934B
:10024000AAE60D911C914AE050E09CD0AAE60D93DD
:100250001C93AAE60D911C9140E150E098D0AAE6CB
:100260004D935C93AFE68C91E0E322D181E08A93D9
:10027000AFE68C916CECBB27A6E1E0E345D181E0D1
:100280008A93AFE68C9164E4BB27A6E1E0E33CD11E
:100290000895ACE68C918F5F8C9300916C000530D3
:1002A00009F003C080E080936C00AEE68C9184FB83
:1002B000882780F9809580FBA2E38C9183F98C9349
:1002C00081E080936D0000916D00033010F009F023
:1002D00026C0A2E60D911C914AE050E07ED0A8E62F
:1002E0000D931C938091680080936400EAE7F3E02B
:1002F000A4E68C919927ADE6AD90A4E6AA0DB3D003
:10030000A2E60D911C914AE050E067D0A2E64D9321
:100310005C93ADE68C918F5F8C9308F4D4CF009101
:100320006700083209F003C08FEF809367000091E7
:100330006C00003009F005C0A7E68C9188BB969848
:100340001BC0013009F008C0969A009166004FED7D
:10035000042308BB959810C0023009F006C0959A96
:10036000A5E68C9188BB949807C0033009F004C0BF
:10037000949A8FEF88BB2ADF089528EB32A2E1A47C
:1003800024EA20A008D043D000FC10D0089503D068
:1003900024D001F8F9CF0024E89457FF02C009D017
:1003A000689400F80BD010F80124089502D009D009
:1003B0000895509540954F5F5F4F0895E89417FF5B
:1003C0000895009510950F5F1F4F68940895992325
:1003D0001AF48095909501960895352F242FE8946E
:1003E000452B11F468940895512F402F00271127B1
:1003F00080E1440F551F001F111F021B130B4160AA
:1004000018F4020F131F4E7F8A9599F70895752FE0
:10041000642F55274427FF93F1E1889405C010F419
:10042000460F571F5695479517950795FA95B9F7B3
:10043000FF9108953197F1F70895689462F808954F
:10044000E89462F80895C89531960020089591E0E7
:1004500005C092E003C094E001C098E0F4DF0D9283
:100460009A95E1F70895E80FF91FF1CF91E08823FD
:1004700021F08894991F8A95E9F7892F909508951E
:100480000181082B018312811923128300000000CF
:10049000000000000000000000000000000000005C
:1004A00000000000000000000000000000000895AF
:1004B000C4DFFF27DBDFE4DFEF93FF93ECEBF3E038
:1004C000B9DFFF91EF91182B128309230183EF937A
:1004D000FF93E0EBF0E0AEDFFF91EF911081182386
:1004E00059F4EF93FF93ECEBF3E0A4DFFF91EF916E
:1004F0001081182309F0A4DFEF93FF93ECEBF3E0F6
:1005000099DFFF91EF910895B1DFFF2729915D9168
:1005100048E0B6DF0000000000000000000000001E
:1005200000000000000000000000000000000000CB
:10053000000000000000579510F4182B1283EF9371
:10054000FF93E4E7F0E076DFFF91EF91182B128341
:10055000000000000000000000000000000000009B
:10056000000000000000000000000000000000008B
:1005700000004A9571F62A9551F6089577DFFF2716
:10058000299148E055277CDF09230183EF93FF93EE
:10059000E8E0F0E04FDFFF91EF918894108118239D
:1005A00009F008945795EF93FF93E6E5F0E042DFFA
:1005B000FF91EF914A9539F75D932A9511F70895C8
:00000001FF
